:1000000018308A00532D0000FF00030E8301A10069
:100010000A08A0008A010408A2007708A300780853
:10002000A4007908A5007A08A6007B08A70083131E
:1000300083128C308400801E1F288C1A32282208DC
:1000400084002308F7002408F8002508F900260892
:10005000FA002708FB0020088A00210E8300FF0E0B
:100060007F0E09008A110A12EF280A108A100A115D
:1000700082074F344E3434344934593420345234A6
:1000800042344F3458342D343334323461344434B0
:10009000573400340A108A100A1182074E344F3444
:1000A0002034573441345234523441344E34543471
:1000B00049344534533420344F34523400340A1018
:1000C0008A100A118207203443344F344D344D34A2
:1000D000453452344334493441344C34203455345B
:1000E00053344534203400340A108A100A11820730
:1000F00020344F34203400340A108A100A11820749
:1001000020344534203400340A108A100A11820742
:100110002034203400340A108A100A118207203457
:10012000533441345434533400340A108A100A11C1
:100130008207483444344F345034203400340A1099
:100140008A100A11820753344534523449344134F9
:100150004C3420344F344B3400340A108A100A11C6
:1001600082074E344F3454342034413420344734E1
:100170005034533400340A108A100A11820747346D
:1001800050345334203446344F3455344E34443490
:1001900000340A108A100A1182074734503452344E
:1001A0004D34433420345034463400340A108A101D
:1001B0000A118207473450344734473441342034DD
:1001C0005034463400340A108A100A1182074E3423
:1001D0004F3420344734503453343F340034831682
:1001E00086108312861428302C0784008C1EF62873
:1001F0001A0880002C088316E900013083122C07AE
:100200000339AC002D082C02031D0A298316690846
:100210008312AC0083168610831286108C128A110A
:100220000A121F28643084000008031926290130AF
:10023000F800F701F70B1A29F80B19296630F700B7
:10024000F70B202900000000800B172900340E3026
:10025000F700F70B292974081039003A031D3229D9
:100260000812332908168316081274082039003A38
:10027000031D3E2983128812402983168312881693
:100280008316881274084039003A031D4B298312E3
:1002900008134D2983168312081783160813740850
:1002A0008039003A031D5829831288135A2983166E
:1002B0008312881783168813881183128815831672
:1002C00088118312881174080139003A031D6A29C4
:1002D00008126B2908168316081274080239003AAE
:1002E000031D7629831288127829831683128816B3
:1002F0008316881274080439003A031D8329831277
:1003000008138529831683120817831608137408A7
:100310000839003A031D9029831288139229831605
:100320008312881783168813881183128815831601
:100330008811831288110034831688108312881064
:100340000830F40027210130F40027210230E400B6
:1003500012210230F40027210230E400122106307D
:10036000F40027210C30F40027210230E400122190
:10037000003483168810831288147308F400272130
:100380000034831688108312881080306B07EC00CD
:10039000F4002721003483161F149F141F159F118A
:1003A00083121F108316091283129412DD125D0846
:1003B0008316870083125D165D08831687008312FB
:1003C000DD115D08831687000030831294008316C8
:1003D00094000108C7390838810083129001003069
:1003E000F800920000308316920083125D155D08BC
:1003F00083168700831297019701DD145D08831629
:10040000870083129D019D0183168C16C0308312D4
:100410008B0483160610831206148316861083122B
:100420008610831606118312061183168611831215
:100430008611831606128312061283168612831201
:1004400086120330E3008316881083128810831607
:1004500088118312881183160811831208110F3036
:10046000E400122163080139003A031D392A0812F9
:100470003A2A081683160812831263080239003AD2
:10048000031D442A8812452A88168316881283126F
:1004900063080439003A031D4F2A0813502A08172D
:1004A00083160813831263080839003A031D5A2A79
:1004B00088135B2A8817831688138811831288157E
:1004C00083168811831288110530E4001221630815
:1004D0000139003A031D6E2A08126F2A0816831686
:1004E0000812831263080239003A031D792A881220
:1004F0007A2A881683168812831263080439003A10
:10050000031D842A0813852A0817831608138312EB
:1005100063080839003A031D8F2A8813902A881728
:100520008316881388118312881583168811831205
:1005300088110530E400122163080139003A031DD7
:10054000A32A0812A42A0816831608128312630825
:100550000239003A031DAE2A8812AF2A8816831684
:100560008812831263080439003A031DB92A08135C
:10057000BA2A081783160813831263080839003A49
:10058000031DC42A8813C52A881783168813881167
:100590008312881583168811831288110530E400B0
:1005A00012210812831608128312881683168812E5
:1005B0008312081383160813831288138316881373
:1005C00088118312881583168811831288112830A8
:1005D000F40027219C21E30163083520003803192A
:1005E000F52AE30AF300B921EC2A0330E300FA30DC
:1005F000E4001221E30BF72A4030EB00C121E301B4
:1006000063084A2000380319092BE30AF300B921D3
:10061000002B83160610831206100230E300FA3016
:10062000E4001221E30B0F2B831606108312061031
:100630004030EB00C121E30163085F20003803195B
:10064000252BE30AF300B9211C2B0230E300FA301A
:10065000E4001221E30B272B8316061083120614E5
:100660008A150A16762D2D082C020319332B2830F3
:100670002D0784000008EB0001302D070339AD0081
:100680006B08F80000346910E801E8016808E80A1E
:10069000003A0319582B63306807EA0033236A08CD
:1006A0008400780880006808033C031C0030462B57
:1006B00069187B2B33237808E7006308473C031D48
:1006C000712B6408503C031D712B6508523C031DBF
:1006D000712B66084D3C031D712B6708433C0319C1
:1006E0006914E80A6408E3006508E4006608E500A8
:1006F0006708E600582B003069180130F800003414
:1007000033237808E40064082C3C03198B2B332333
:100710007808E400832B0034332333237808AE00B9
:1007200033237808AF0033237808B00033237808E8
:10073000B10033237808B20033237808B3000230C5
:10074000B30730303302093C0318A92B0A30B30237
:10075000B20A30303202053C0318B12B3030B200FF
:10076000B10A30303102093C0318B92B0A30B1020A
:10077000B00A30303002053C0318C12B3030B000D5
:10078000AF0A802333237808413C031DC92B5C1436
:10079000CA2B5C10802333237808B40033237808F5
:1007A000B50033237808B60033237808B700332325
:1007B00033237808B8008023802333237808B900D6
:1007C00033237808BA0033237808BB003323780832
:1007D000BC0033237808BD00802333237808BE0093
:1007E00080238023802333237808BF0033237808B5
:1007F000C00033237808C10033237808C2008A156B
:100800000A16262EF701F801700803107118F70771
:10081000F70CF80CF118F707F70CF80C7119F7073B
:10082000F70CF80CF119F707F70CF80C711AF70729
:10083000F70CF80CF11AF707F70CF80C711BF70717
:10084000F70CF80CF11BF707F70CF80C00348E309E
:10085000F70083165308F8005208F900FA01F80867
:10086000031D3C2C7908F800F9010830F702F8085C
:10087000031D3C2CF701442C0310F81B432CF90DED
:10088000F80DF7033C2CF81300008312003480307D
:10089000831C4D2C8316D80683128316DD01DE01DE
:1008A0005408DC005808DC0653080319382DDB0017
:1008B000F70057080319412DDB020319DE2C031C36
:1008C0009D2C5808E100E1175908E0005A08DF00A4
:1008D000DE010310E10CE00CDF0CDE0CDB0B682CFE
:1008E000DC1F752C5D14552D5D105B105D16D63028
:1008F00084006A2D5D12DC1B872C5B1C922CE10CA2
:10090000E00CDF0CDE0CF70A0319502D922CE11BD2
:10091000952C0310DE0DDF0DE00DE10DF70303193B
:10092000502D872C5D17FD2C5D135408DC00D41F5F
:100930009B2CE117492DE113492D5708DB00F700E7
:100940005308DB025408E100E1175508E00056089F
:10095000DF00DE010310E10CE00CDF0CDE0CDB0B32
:10096000A92CDC1FB62CDD14552DDD105B10DD1617
:10097000DA3084006A2DDD12DC1BC82C5B1CD32C02
:10098000E10CE00CDF0CDE0CF70A0319502DD32C20
:10099000E11BD62C0310DE0DDF0DE00DE10DF7039A
:1009A0000319502DC82CDD17FD2CDD135808DC0071
:1009B000D81FDC2CE117492DE113492D5808E1001F
:1009C000E1175908E0005A08DF00DC1FEB2CE113A7
:1009D0005D15552D5D11DE015B10D63084006A2D4A
:1009E000DC1B132D5408DC005B1CFD2CE10CE00C1F
:1009F000DF0CDE0CF70A0319502DDE1F0E2DDF0A67
:100A0000031D0E2DE00A031D0E2DE10A031D0E2D00
:100A1000E10CE00CDF0CF70A0319502D5D1B942C40
:100A2000DD1BD52C322D8030E106E11F1B2D552D0D
:100A30005808DC00282D5408DC00E108031D282D8F
:100A4000E008031D282DDF08031D282DF701492D7F
:100A5000E11B322D0310DE0DDF0DE00DE10DF70B74
:100A6000282D502DDC1F362DE117492DE113492D7E
:100A70005708F7005808E1005908E0005A08DF005D
:100A8000492D5308F7005408E1005508E0005608C6
:100A9000DF006108F8006008F9005F08FA00882D9F
:100AA000F701F801F901FA01882DDE01DF09E009FB
:100AB000E109DE09DE0A031D632DDF0A031D632D34
:100AC000E00A0319E10A5D18742CDD18B52C5D19D4
:100AD000EA2C182D0008DF07031C742DE00A031D03
:100AE000742DE10A03195B1484030008E007031C5A
:100AF0007C2DE10A03195B1484030008801F803AEF
:100B0000E10703185B145D1A7A2CDD1ABB2CF02C5C
:100B100000008312003483164E080319512EDA00A8
:100B200052080319512EDA02031C9B2D7F30DA077D
:100B30000318512EA12D8130DA02031C512E031906
:100B4000512E5A08F700F801F901FA01D9014F08AE
:100B5000D800D8175008D7005108D6001930DA004D
:100B60005508D6020318C42D0130D7020318C42D2E
:100B7000D8020318C42DD9020318C42DD90AD80AE3
:100B8000D70A5508D607F62D5408D7020318DF2DCB
:100B90000130D8020318DF2DD9020318DF2DD90A3E
:100BA000D80A5408D7075508D607031CF62DD70ACC
:100BB000031DF62DD80A031DF62DD90AF62D53086C
:100BC0008038D8020318F52D0130D9020318F52D0D
:100BD000D90A53088038D8075408D707031CD32DE7
:100BE000D80A031DD32DD90AD32D7A14DA0BF92D87
:100BF000042E0310D60DD70DD80DD90D0310FA0D04
:100C0000F90DF80DDB0DB02D5B1C0C2E0310F80C4C
:100C1000F90CFA0CDB0C0F2EF7030319512EDB1B1A
:100C2000382E0310D60DD70DD80DD90D5508D60284
:100C30000318242E0130D7020318242ED8020318DB
:100C4000242ED902031C472E5408D70203182F2E36
:100C50000130D80203182F2ED902031C472E530847
:100C60008038D8020318382E0130D902031C472ED1
:100C7000FA0A031D472EF90A031D472EF80A031D21
:100C8000472EF70A0319512EF80CF90CFA0C4F08ED
:100C9000DA005308DA06DA1F4F2EF817552EF8132C
:100CA000552EF701F801F901FA0100008312003412
:100CB000831652080319C92EDA0056080319C92EE3
:100CC000DA0703186A2E7F30DA02031CC92E0319D3
:100CD000C92E6E2E8130DA070318C92E5A08F70084
:100CE000F801F901FA015308DE00DE175408DD00AF
:100CF0005508DC001830DA00DB015C1C972E59081F
:100D0000FA07031C892EF90A031D892EF80A031914
:100D1000DB175808F907031C902EF80A0319DB1794
:100D20005708D400D4175408F8070318DB17DB0D55
:100D3000F80CF90CFA0CDE0CDD0CDC0C0310DA0BF1
:100D40007C2E0130F7070318C92EF81BAE2EDE0DDE
:100D5000FA0DF90DF80DF7030319C92EDE1FBF2E8A
:100D6000FA0A031DBF2EF90A031DBF2EF80A031D40
:100D7000BF2EF80CF90CFA0CF70A0319C92E530808
:100D8000DB005708DB06DB1FC72EF817CD2EF81344
:100D9000CD2EF701F801F901FA01000083120034A9
:100DA00083164F08D6005308D606D61FDC2E031133
:100DB0000310CF1B03140F2F4F08D6005208D70083
:100DC0004E08D7020319EA2ED61F0F2F0308013A47
:100DD00083000F2F5308D7004F08D7020319F62EB0
:100DE000D61F0F2F0308013A83000F2F5408D70096
:100DF0005008D7020319022FD61F0F2F0308013AFC
:100E000083000F2F5508D7005108D70203190E2F62
:100E1000D61F0F2F0308013A83000F2F03108312F0
:100E200000348E30F70083164E08F7024F08F900A1
:100E30005008F800F917F7080319292F0310F908CB
:100E4000031D252FF8080319292FF90CF80CF70BAF
:100E50001E2FCF1F302FF809F909F80A0319F90AD4
:100E6000000083120034831483162308D60022085E
:100E7000D5002108D4002008D300DB30DA000F3081
:100E8000D9004930D8007F30D70083124724770833
:100E90008316A4007808A5007908A6007A08A700A0
:100EA000AB002608AA002508A9002408A8008A1576
:100EB000831258218A1100347208F8017102031854
:100EC000642F7108F700702FF7010830F300F10D5F
:100ED000F70D720877020318F700F80DF30B672F70
:100EE00000341030F700FA01EF01EC0CEB0C031C9E
:100EF0007F2F6D08FA070318EF0A6E08EF07EF0C53
:100F0000FA0CF90CF80CF70B752F8A110A16FD284C
:100F1000F801F901F701FA016C08031D922F6B0823
:100F20000319AC2F1030ED000310E90DEA0DF70D99
:100F3000FA0D6C087A02031D9F2F6B087702031CC1
:100F4000A82F6B08F702031CFA036C08FA020314BB
:100F5000F80DF90DED0B942F00008A110A16E42903
:100F60006910E801E8016808E80A003A0319C52F8A
:100F700063306807EA0033236A0884007808800039
:100F80006808033C031C0030B32F6918E82F332393
:100F90007808E7006308473C031DDE2F6408503CD7
:100FA000031DDE2F6508473C031DDE2F6608473C06
:100FB000031DDE2F6708413C03196914E80A640821
:100FC000E3006508E4006608E5006708E600C52F51
:0E0FD000003069180130F8008A150A16602EEC
:1010000030304102E800F0000A30F1008A11022479
:101010008A157808E900303042026907E300303071
:101020003F02E800F0000A30F1008A1102248A151C
:101030007808E900303040026907E4006308013AAB
:1010400003194428033A03194828013A03194D2883
:10105000073A03195228013A03195728033A03198A
:101060005C28013A031961280F3A03196628013AEE
:1010700003196B28033A03197328013A03197B28D3
:10108000073A031983288B28E6016408E5008E28B7
:101090001F306407E500E6018E283B306407E50059
:1010A000E6018E285A306407E500E6018E28783084
:1010B0006407E500E6018E2897306407E500E60145
:1010C0008E28B5306407E500E6018E28D430640729
:1010D000E500E6018E28E6016408E500F330E50747
:1010E0000318E60A8E2811306407E5000130E60097
:1010F0000318E60A8E2830306407E5000130E60068
:101100000318E60A8E284E306407E5000130E60039
:101110000318E60A8E28E6010130E50030302E0281
:10112000E800F0000A30F1008A1102248A157808DC
:10113000E90030302F0269078316D301D2008A11EB
:10114000831227248A157A08D1007908D0007808FC
:10115000CF007708CE0001306502E7006608E8009E
:101160000030031C0130E802831451088316D600B6
:10117000831250088316D50083124F088316D400BB
:1011800083124E088316D300DA01D9014030D8000B
:101190008230D7008A11831247248A157708E90024
:1011A0007808EA007908EB007A08EC008316D10091
:1011B00083126B088316D00083126A088316CF004F
:1011C000831269088316CE00D501D4014030D300C4
:1011D0008330D2008A1183128B258A157708ED009F
:1011E0007808EE007908EF007A08F00068088316A6
:1011F000D300831267088316D2008A118312272432
:101200008A1583107A088316D6007908D5007808E5
:10121000D4007708D3007008DA0083126F088316B1
:10122000D90083126E088316D80083126D088316C6
:10123000D7008A11831247248A157708F1007808AD
:10124000F2007908F3007A08F4008316D1007308DD
:10125000D0007208CF007108CE00D5018030D400D4
:101260003630D3008730D2008A1183128B258A153D
:10127000DB308316D5000F30D4004930D3008130E5
:10128000D2007A08D9007908D8007808D700770802
:10129000D6008A11831258268A157A08D100790857
:1012A000D0007808CF007708CE008A150A163F2EA6
:1012B0007F308316B400B501B601B7017E30BE00A1
:1012C0008030BF00C001C1017A30C2002A30C300A3
:1012D000AA30C400A330C5007530C600B630C700C0
:1012E0000930C8009C30C9006F30CA004F30CB00B5
:1012F000B430CC000B30CD002B08D1002A08D00030
:101300002908CF002808CE00D501D401D301D2018D
:101310008A118312D0268A15031C922980308316E5
:10132000A906831283162B08D1002A08D0002908A9
:10133000CF002808CE00DB30D5000F30D400493074
:10134000D3007F30D2008A1183128B258A157A0848
:101350008316D1007908D0007808CF007708CE0036
:101360008A11831211278A1578088316B8002B0872
:10137000D1002A08D0002908CF002808CE00DB3091
:10138000D5000F30D4004930D3007F30D2008A110D
:1013900083128B258A1577088316CE007808CF0034
:1013A0007908D0007A08D100D3013808D2008A1118
:1013B000831227248A15831483165108D6005008F7
:1013C000D5004F08D4004E08D3007A08DA00790817
:1013D000D9007808D8007708D7008A1183124724EB
:1013E0008A157A088316BD007908BC007808BB000E
:1013F0007708BA000330B805B8080319032A38087B
:10140000023C031D212A3D08D5003C08D4003B08BE
:10141000D3003A08D200DB30D9000F30D800493071
:10142000D7007F30D6008A11831258268A157A0891
:101430008316B3007908B2007808B1007708B000CD
:10144000922A380B5B2A8314D601D501D4017F3050
:10145000D3003D08DA003C08D9003B08D8003A0820
:10146000D7008A11831247248A1577088316CE0085
:101470007808CF007908D0007A08D100D50050084C
:10148000D4004F08D3004E08D200DB30D9000F3013
:10149000D8004930D7007F30D6008A1183125826F1
:1014A0008A157A088316B3007908B2007808B1006B
:1014B0007708B000922A83143D08D6003C08D50076
:1014C0003B08D4003A08D300DA01D901D8017F30B3
:1014D000D7008A11831247248A1577088316CE0015
:1014E0007808CF007908D0007A08D100D5005008DC
:1014F000D4004F08D3004E08D200DB30D9000F30A3
:10150000D8004930D7007F30D6008A118312582680
:101510008A157A088316B3007908B2007808B100FA
:101520007708B000AF01AE01AD017F30AC003308E9
:10153000D5003208D4003108D3003008D200330877
:10154000D9003208D8003108D7003008D6008A11F7
:10155000831258268A157A088316B3007908B200D8
:101560007808B1007708B000B9013908033C031CC2
:10157000212B3708D5003608D4003508D3003408AD
:10158000D2003308D9003208D8003108D70030081B
:10159000D6008A11831258268A157A088316B70056
:1015A0007908B6007808B5007708B400390DF7005F
:1015B000F70DFC30F7057708BE3E84000008CE002A
:1015C000840A0008CF00840A0008D000840A0008BA
:1015D000D100D5005008D4004F08D3004E08D200E7
:1015E0003708D9003608D8003508D7003408D600A7
:1015F0008A11831258268A1504088316D200831094
:101600002F08D6002E08D5002D08D4002C08D300B2
:101610007A08DA007908D9007808D8007708D70066
:101620008A11831247248A158316520884007A0887
:10163000AF007908AE007808AD007708AC00B90AB1
:10164000B52A3808023C0319272B380B292B803088
:10165000AD062C08F7002D08F8002E08F9002F0819
:10166000FA008312003451088316AB00831250082D
:101670008316AA0083124F088316A90083124E080E
:101680008316A800831258217A08E6007908E5003D
:101690007808E4007708E30051088316A30083125A
:1016A00050088316A20083124F088316A1008312EC
:1016B0004E088316A0008A11831233278A157A08F0
:1016C000EA007908E9007808E8007708E70051089F
:1016D0008316D500831250088316D40083124F0856
:1016E0008316D30083124E088316D200D901D80185
:1016F000D7018030D6008A11831258268A157708C0
:10170000F3007808F4007908F5007A08F6008316EB
:10171000AB007508AA007408A9007308A80083121A
:1017200058217A08EE007908ED007808EC00770877
:10173000EB0051088316D500831250088316D4009D
:1017400083124F088316D30083124E088316D200EB
:10175000D901D801D7018030D6008A1183125826CA
:101760008A157708F3007808F4007908F5007A08FC
:10177000F6008316A3007508A2007408A100730880
:10178000A0008A11831233278A157A08F20079089B
:10179000F1007808F0007708EF005230D5004930AA
:1017A000D4001D30D3007130D200AE308316D50086
:1017B000D730D4007430D3007530D200831266085D
:1017C0008316D900831265088316D8008312640833
:1017D0008316D700831263088316D6008A118312FA
:1017E00058268A15831055088316D600831254088C
:1017F0008316D500831253088316D400831252082F
:101800008316D3007A08DA007908D9007808D8005E
:101810007708D7008A11831247248A157A08D500E1
:101820007908D4007808D3007708D2002C308316CA
:10183000D5006330D4000330D3007A30D200831255
:101840006A088316D900831269088316D8008312A8
:1018500068088316D700831267088316D6008A119A
:10186000831258268A15831455088316D6008312CE
:1018700054088316D500831253088316D4008312AC
:1018800052088316D3007A08DA007908D90078085C
:10189000D8007708D7008A11831247248A157A085E
:1018A000D5007908D4007808D3007708D200C13079
:1018B0008316D5007330D4006F30D3007830D20057
:1018C00083126E088316D90083126D088316D80020
:1018D00083126C088316D70083126B088316D60018
:1018E0008A11831258268A15831455088316D60048
:1018F000831254088316D500831253088316D4002C
:10190000831252088316D3007A08DA007908D900C6
:101910007808D8007708D7008A11831247248A15DF
:101920007A08D5007908D4007808D3007708D20067
:1019300048308316D5005130D4002730D3007A3098
:10194000D2007208D9007108D8007008D70083123D
:101950006F088316D6008A11831258268A158314BD
:1019600055088316D600831254088316D5008312B7
:1019700053088316D400831252088316D3007A08C2
:10198000DA007908D9007808D8007708D7008A11DA
:10199000831247248A157A08D5007908D40078087C
:1019A000D3007708D20055088316D5008312540857
:1019B0008316D400831253088316D300831252086F
:1019C0008316D2001430D9002E30D8006530D700ED
:1019D0008630D6008A11831258268A157A08D500D7
:1019E0007908D4007808D3007708D2008A150A163F
:1019F000422E51088316AB00831250088316AA00AA
:101A000083124F088316A90083124E088316A8007C
:101A1000831258217A08E6007908E5007808E40086
:101A20007708E30051088316A30083125008831639
:101A3000A20083124F088316A10083124E0883165A
:101A4000A0008A11831233278A157A08EA007908E0
:101A5000E9007808E8007708E70051088316D50008
:101A6000831250088316D40083124F088316D300C4
:101A700083124E088316D200D901D801D7018030D5
:101A8000D6008A11831258268A157708F300780841
:101A9000F4007908F5007A08F6008316AB0079089F
:101AA000AA007808A9007708A800831258217A08AC
:101AB000EE007908ED007808EC007708EB0051089B
:101AC0008316D500831250088316D40083124F0862
:101AD0008316D30083124E088316D200D901D80191
:101AE000D7018030D6008A11831258268A157708CC
:101AF000F3007808F4007908F5007A08F6008316F8
:101B0000A3007908A2007808A1007708A0008A1134
:101B1000831233278A157A08F2007908F1007808D1
:101B2000F0007708EF006430D900B030D8006230A0
:101B3000D7007730D60044308316D500C130D400AA
:101B40004C30D3007D30D200831266088316D90052
:101B5000831265088316D800831264088316D700A1
:101B6000831263088316D6008A11831258268A15B9
:101B7000831459088316D600831258088316D5009B
:101B8000831257088316D400831256088316D30095
:101B90007A08DA007908D9007808D8007708D700E1
:101BA0008A11831247248A157A08D9007908D80047
:101BB0007808D7007708D600E7308316D500E230E2
:101BC000D4000F30D3007B30D20083126A08831612
:101BD000D900831269088316D80083126808831617
:101BE000D700831267088316D6008A1183125826FD
:101BF0008A15831059088316D60083125808831655
:101C0000D500831257088316D40083125608831612
:101C1000D3007A08DA007908D9007808D800770864
:101C2000D7008A11831247248A157A08D9007908C7
:101C3000D8007808D7007708D60036308316D5004C
:101C40007230D4005D30D3007730D20083126E083A
:101C50008316D90083126D088316D80083126C088E
:101C60008316D70083126B088316D6008A1183125D
:101C700058268A15831459088316D60083125808EB
:101C80008316D500831257088316D4008312560892
:101C90008316D3007A08DA007908D9007808D800CA
:101CA0007708D7008A11831247248A157A08D90049
:101CB0007908D8007808D7007708D600BD30831699
:101CC000D500C330D4006D30D3007430D200720818
:101CD000D9007108D8007008D70083126F088316E6
:101CE000D6008A11831258268A1583105908831644
:101CF000D600831258088316D5008312570883161E
:101D0000D400831256088316D3007A08DA007908C3
:101D1000D9007808D8007708D7008A1183124724A1
:101D20008A157A08D9007908D8007808D70077088A
:101D3000D6008316D501D4014030D3008030D200C4
:101D4000831251088316D900831250088316D800D5
:101D500083124F088316D70083124E088316D600CD
:101D60008A11831258268A157708F3007808F40040
:101D70007908F5007A08F6008316AB007908AA0006
:101D80007808A9007708A800831258212730831605
:101D9000D500C030D4003030D3007630D2007A087D
:101DA000D9007908D8007808D7007708D6008A11BA
:101DB000831258268A150408F400831459088316E0
:101DC000D600831258088316D5008312570883164D
:101DD000D400831256088316D3007A08DA007908F3
:101DE000D9007808D8007708D7008A1183124724D1
:101DF0008A15740884007A08D9007908D800780810
:101E0000D7007708D6008316D501D4014030D3001F
:101E10008030D200831251088316D90083125008F3
:101E20008316D80083124F088316D70083124E08FA
:101E30008316D6008A11831258268A157708F30074
:101E40007808F4007908F5007A08F6008316A300F4
:101E50007908A2007808A1007708A0008A118312EF
:101E600033278A158F308316D500FC30D4004130DB
:101E7000D3007530D2007A08D9007908D8007808E4
:101E8000D7007708D6008A11831258268A150408CD
:101E9000F400831059088316D6008312580883165D
:101EA000D500831257088316D40083125608831670
:101EB000D3007A08DA007908D9007808D8007708C2
:101EC000D7008A11831247248A15740884007A087F
:101ED000D9007908D8007808D7007708D6008A1585
:101EE0000A16452E51088316D10083125008831616
:101EF000D00083124F088316CF0083124E0883163A
:101F0000CE00D501D401D3018130D2008A118312D1
:101F10008B258A157708E3007808E4007908E50046
:101F20007A08E600831466088316D60083126508D3
:101F30008316D500831264088316D40083126308C5
:101F40008316D300DA01D9013430D8008630D700A7
:101F50008A11831247248A157708E7007808E80079
:101F60007908E9007A08EA008316D5008312690827
:101F70008316D400831268088316D300831267087F
:101F80008316D200DB30D9000F30D8004930D7009B
:101F90008030D6008A11831258268A157708EB0004
:101FA0007808EC007908ED007A08EE008316D1007D
:101FB00083126D088316D00083126C088316CF003D
:101FC00083126B088316CE00D501D4013430D300C0
:101FD0008630D2008A1183128B258A157A08D100A7
:101FE0007908D0007808CF007708CE008A150A1645
:021FF0004B2E76
:1020000030302E02EC00F0000A30F1000A120224F7
:102010000A167808ED0030302F026D07E700E8015E
:1020200030303002EC00F0000A30F1000A120224D5
:102030000A167808ED00303031026D07E9003030C3
:102040003902EC00F0006430F1000A1202240A1692
:102050007808ED0030303A02EF00F0000A30F1006D
:102060000A1202240A1678086D07F00030303B028D
:1020700070078316D301D2000A12831227240A168E
:102080007A08E6007908E5007808E4007708E300BC
:1020900030303C02EC00F0000A30F1000A12022459
:1020A0000A163D087807D03EF000F1003C30F200FF
:1020B0000A125C270A1678088316D301D2000A1286
:1020C000831227240A16831066088316D60083120B
:1020D00065088316D500831264088316D400831222
:1020E00063088316D3007A08DA007908D9007808E3
:1020F000D8007708D7000A12831247240A167A08F4
:10210000E6007908E5007808E4007708E3003E0877
:10211000573C031DAE288316D501D4018030D3006F
:102120007F30D200831266088316D90083126508B7
:102130008316D800831264088316D70083126308BD
:102140008316D6000A12831258260A167A08E60069
:102150007908E5007808E4007708E3008316D501E4
:10216000D401D3018130D200831266088316D900CE
:10217000831265088316D800831264088316D7007B
:10218000831263088316D6000A12831258260A1691
:10219000831055088316D600831254088316D50081
:1021A000831253088316D400831252088316D30077
:1021B0007A08DA007908D9007808D8007708D700BB
:1021C0000A12831247240A167A08D1007908D0002F
:1021D0007808CF007708CE005108E6005008E500E7
:1021E0004F08E4004E08E3006808EC006708EB00C5
:1021F000EE013C30ED000A12712F0A167908FA0040
:1022000078088316D2007908D3000A128312272493
:102210000A16831066088316D60083126508831693
:10222000D500831264088316D400831263088316D2
:10223000D3007A08DA007908D9007808D80077083E
:10224000D7000A12831247240A167708EB00780891
:10225000EC007908ED007A08EE008316D3018312B2
:1022600069088316D2000A12831227240A168310E3
:102270006E088316D60083126D088316D50083126C
:102280006C088316D40083126B088316D3007A0877
:10229000DA007908D9007808D8007708D7000A1240
:1022A000831247240A167A08D1007908D0007808EA
:1022B000CF007708CE0051088316D1008312500852
:1022C0008316D00083124F088316CF0083124E0866
:1022D0008316CE00D501D4013430D3008830D2002B
:1022E0000A128312D0260A16031C7829DC147929D5
:1022F000DC108A150A16482E30303402E800F0004F
:102300000A30F1000A1202240A167808E900303077
:10231000350269078316D301D2000A1283122724DB
:102320000A167A08E6007908E5007808E4007708DC
:10233000E30030303602E800F0000A30F1000A1203
:1023400002240A1637087807D03EEC00F1003C3032
:10235000F2000A125C270A1678088316D301D2000D
:102360000A12831227240A16831066088316D600E1
:10237000831265088316D500831264088316D4007F
:10238000831263088316D3007A08DA007908D9002B
:102390007808D8007708D7000A12831247240A1653
:1023A0007A08E6007908E5007808E4007708E30099
:1023B00030303802E800EA016808E9000230EC0039
:1023C0005830EB000A12882F0A167908FA007808AC
:1023D0008316D2007908D3000A12831227240A1622
:1023E000831066088316D600831265088316D5000D
:1023F000831264088316D400831263088316D30003
:102400007A08DA007908D9007808D8007708D70068
:102410000A12831247240A167A08E6007908E500B2
:102420007808E4007708E30066088316D500831275
:1024300065088316D400831264088316D3008312C0
:1024400063088316D200DB30D9000F30D800493042
:10245000D7008030D6000A12831258260A16770851
:10246000E7007808E8007908E9007A08EA008316AE
:10247000D100831269088316D0008312680883167E
:10248000CF00831267088316CE00D501D401343003
:10249000D3008630D2000A1283128B250A167A08DE
:1024A000E6007908E5007808E4007708E3006608AC
:1024B000D5006508D4006408D3006308D200510831
:1024C0008316AB00831250088316AA0083124F08AC
:1024D0008316A90083124E088316A8000A128A15D3
:1024E000831258210A168A117A08D1007908D0007F
:1024F0007808CF007708CE0066088316AB008312F9
:1025000065088316AA00831264088316A900831243
:1025100063088316A8000A128A15831258210A1626
:102520008A117708E7007808E8007908E9007A0856
:10253000EA0059088316AB00831258088316AA00D4
:10254000831257088316A900831256088316A80021
:102550000A128A15831258210A168A116A088316EC
:10256000D500831269088316D40083126808831685
:10257000D300831267088316D2007A08D90079083D
:10258000D8007808D7007708D6000A128312582698
:102590000A167708EB007808EC007908ED007A0855
:1025A000EE008316D50083126D088316D4008312C3
:1025B0006C088316D30083126B088316D200831233
:1025C00051088316D900831250088316D80083124D
:1025D0004F088316D70083124E088316D6000A12BE
:1025E000831258260A167A08D1007908D000780894
:1025F000CF007708CE0066088316A3008312650813
:102600008316A200831264088316A1008312630854
:102610008316A0000A12831233270A167708E700F0
:102620007808E8007908E9007A08EA005908831672
:10263000A300831258088316A2008312570883163A
:10264000A100831256088316A0000A1283123327B2
:102650000A166A088316D500831269088316D40007
:10266000831268088316D300831267088316D2008A
:102670007A08D9007908D8007808D7007708D600FA
:102680000A12831258260A160408EB008310510818
:102690008316D600831250088316D50083124F0884
:1026A0008316D40083124E088316D3007A08DA000A
:1026B0007908D9007808D8007708D7000A12831261
:1026C00047240A166B0884007A08D1007908D000E4
:1026D0007808CF007708CE008A150A164E2E6A08B1
:1026E000F2006908F1006808F0006708EF000130A7
:1026F000F300741072088316A3007108A20070081A
:10270000A10083126F088316A0007208D10071081F
:10271000D0007008CF0083126F088316CE00D50159
:10272000D401D301D2010A128312D0260A16031C47
:102730009E2B741480308316A10683128316D10158
:10274000D001CF017E30CE002308D5002208D4006E
:102750002108D3002008D2000A128312D0260A16BC
:10276000031C962C83148316D601D501D4017F3027
:10277000D3002308DA002208D9002108D800200855
:10278000D7000A12831247240A1677088316B0006E
:102790007808B1007908B2007A08B3003308D10094
:1027A0003208D0003108CF003008CE00D501D40166
:1027B000D3018030D2000A1283128B250A167708C3
:1027C0008316B4007808B5007908B6007A08B70017
:1027D0003708BC003608BB003508BA003408B90019
:1027E0003C08D1003B08D0003A08CF003908CE00A1
:1027F000D501D401D301D2010A128312D0260A16C0
:102800000318042C031D092CF701F801F901FA0142
:102810008A2C83163C08C0003B08BF003A08BE0063
:102820003908BD00BD30C500450884000008C80156
:10283000C7007F304707C9004808CA000318CA0A02
:1028400003104A0CFA00490CF900CB00450884003B
:102850004B0880004008C4003F08C3003E08C20087
:102860003D08C1003C08D1003B08D0003A08CF0029
:102870003908CE004008D5003F08D4003E08D300F8
:102880003D08D2000A1283128B250A168310831684
:102890004008D6003F08D5003E08D4003D08D300CC
:1028A0007A08DA007908D9007808D8007708D700C4
:1028B0000A12831247240A167A088316C000790880
:1028C000BF007808BE007708BD004508840080037B
:1028D0004408D1004308D0004208CF004108CE0090
:1028E0004008D5003F08D4003E08D3003D08D20080
:1028F0000A128312D0260A160319802C83162A2C5A
:1029000083164108F7004208F8004308F90044081C
:10291000FA0083127A088316A3007908A2007808C7
:10292000A1007708A0000230F30783128316230862
:10293000D5002208D4002108D3002008D2002308A3
:10294000D9002208D8002108D7002008D6000A1292
:10295000831258260A167A088316AF007908AE004B
:102960007808AD007708AC003730D500BF30D40010
:102970007D30D300D2002F08D9002E08D8002D08B2
:10298000D7002C08D6000A12831258260A16770898
:102990008316B0007808B1007908B2007A08B30055
:1029A00083103308D6003208D5003108D40030082F
:1029B000D3003D30DA00AA30D9009330D8008130FE
:1029C000D7000A12831247240A167A088316A70032
:1029D0007908A6007808A5007708A4002708D50084
:1029E0002608D4002508D3002408D2002F08D900D7
:1029F0002E08D8002D08D7002C08D6000A12831202
:102A000058260A1677088316B0007808B1007908AE
:102A1000B2007A08B30083103308D6003208D5001C
:102A20003108D4003008D300EE30DA005030D9003D
:102A30003330D8008130D7000A12831247240A1697
:102A40007A088316A7007908A6007808A5007708F9
:102A5000A400D501D401D3017F30D2002F08D900C2
:102A60002E08D8002D08D7002C08D6000A12831291
:102A700058260A1677088316B0007808B10079083E
:102A8000B2007A08B30083103308D6003208D500AC
:102A90003108D4003008D3000A30DA008D30D90074
:102AA000B130D8008130D7000A12831247240A16A9
:102AB0007A088316AB007908AA007808A90077087D
:102AC000A8002B08D5002A08D4002908D30028081C
:102AD000D2002F08D9002E08D8002D08D7002C08C6
:102AE000D6000A12831258260A1677088316B000F9
:102AF0007808B1007908B2007A08B300831033086F
:102B0000D6003208D5003108D4003008D300EE30AA
:102B1000DA005030D9003330D8008130D7000A12A3
:102B2000831247240A167A088316AB007908AA0094
:102B30007808A9007708A8002308D5002208D40047
:102B40002108D3002008D2002708D9002608D80081
:102B50002508D7002408D6000A12831258260A1620
:102B600077088316B0007808B1007908B2007A08B7
:102B7000B300D1003208D0003108CF003008CE00B9
:102B80002B08D5002A08D4002908D3002808D20031
:102B90000A1283128B250A167A088316A700790871
:102BA000A6007808A5007708A400F31C072ED5011D
:102BB000D401D3018030D2002708D9002608D800DC
:102BC0002508D7002408D6000A12831258260A16B0
:102BD0008314DB308316D6000F30D5004930D40083
:102BE0007F30D3007A08DA007908D9007808D80055
:102BF0007708D7000A12831247240A167A08831628
:102C0000A7007908A6007808A5007708A400741C1E
:102C10000B2E8030A506731C2B2E8314DB30D600C0
:102C20000F30D5004930D4007F30D3002708DA00B8
:102C30002608D9002508D8002408D7000A128312D4
:102C400047240A167A088316A7007908A600780890
:102C5000A5007708A4002408F7002508F800260836
:102C6000F9002708FA007A088312EE007908ED00CF
:102C70007808EC007708EB006B08F7006C08F800A8
:102C80006D08F9006E08FA0000345108EA00500897
:102C9000E9004F08E8004E08E7006F237A08D100EA
:102CA0007908D0007808CF007708CE008314DB3095
:102CB0008316D6000F30D5004930D4007F30D300C2
:102CC000831251088316DA00831250088316D90044
:102CD00083124F088316D80083124E088316D7003C
:102CE0000A12831247240A167708E7007808E800DA
:102CF0007908E9007A08EA008316D100831279087E
:102D00008316D000831278088316CF0083127708C9
:102D10008316CE00DB30D5000F30D4004930D3000D
:102D20008030D2000A1283128B250A167708EB0036
:102D30007808EC007908ED007A08EE008316D500DB
:102D4000831279088316D400831278088316D3007F
:102D5000831277088316D200D901D8013430D70006
:102D60008630D6000A12831258260A167708EF001A
:102D70007808F0007908F1007A08F20083107A08E8
:102D80008316D6007908D5007808D4008312770816
:102D90008316D300DA01D901D8017E30D7000A1298
:102DA000831247240A167A088316D1007908D000C6
:102DB0007808CF007708CE000A12831211270A166E
:102DC0007808CD008A150A16512EEB010A12C1218E
:102DD0000A163F08F3000A12B9210A164008F30048
:102DE0000A12B9210A162F30F3000A12B9210A1665
:102DF0004108F3000A12B9210A164208F3000A1228
:102E0000B9210A16303031020139013C031D1B2F54
:102E1000E30163080A1274200A1600380319162FFA
:102E2000E30AF3000A12B9210A16092F83160612C3
:102E3000831206162D2FE30163080A127C200A165E
:102E400000380319292FE30AF3000A12B9210A16E0
:102E50001C2F83160612831206122E08F3000A1284
:102E6000B9210A162F08F3000A12B9210A163A30BE
:102E7000F3000A12B9210A163008F3000A12B92128
:102E80000A163108F3000A12B9210A163A30F30083
:102E90000A12B9210A163208F3000A12B9210A16D9
:102EA0003308F3000A12B9210A162030F3000A127F
:102EB000B9210A168A150A16552EE3010A12332380
:102EC0000A166308043C031C6A2F0A1280230A16A0
:102ED000E30A612F0A1233230A1630307802C70042
:102EE0000A1233230A160A1233230A167808C80076
:102EF0000A1233230A167808C900C7080319F72FE6
:102F00000A1233230A167808C3000A1233230A165A
:102F10007808C5000A1233230A167808C600460846
:102F20002E3C031D972F4508C6003030C5004508CC
:102F3000303C031DA52F4608393C031DA42F30301B
:102F4000C6003130C500A52FC60A30304502E40066
:102F50000A30F0006408F1000A1202240A16780808
:102F6000E500303046026507CA000A1280230A16BF
:102F70000A1233230A167808C3000A1233230A16EA
:102F80007808C4000A1233230A167808C5000A120A
:102F900033230A167808C60043082E3C031DD62F9B
:102FA0003030C6002030C500C400C30044082E3CA9
:102FB000031DE02F4308C6002030C500C400C30035
:102FC00045082E3C031DEB2F4408C6004308C500EE
:102FD0002030C400C30046082E3C031DF72F4508CF
:102FE000C6004408C5004308C4002030C3008A1549
:042FF0000A168A2E05
:1030000055088316A300831254088316A200831266
:1030100053088316A100831252088316A0000A12D7
:103020008A11831233270A168A157708E700780871
:10303000E8007908E9007A08EA0051088316AB0035
:10304000831250088316AA0083124F088316A90022
:1030500083124E088316A8000A12831258210A16FA
:103060006A088316D500831269088316D400831278
:1030700068088316D300831267088316D2007A0883
:10308000D9007908D8007808D7007708D6000A1246
:103090008A11831258260A168A157708EB007808D9
:1030A000EC007908ED007A08EE0059088316A300B9
:1030B000831258088316A200831257088316A100B2
:1030C000831256088316A0000A128A11831233272E
:1030D0000A168A150408EF0083146E088316D600BA
:1030E00083126D088316D50083126C088316D400F2
:1030F00083126B088316D3007A08DA007908D900A6
:103100007808D8007708D7000A128A11831247245A
:103110000A168A156F0884007A08D9007908D80041
:103120007808D7007708D60051088316A3008312C9
:1031300050088316A20083124F088316A100831241
:103140004E088316A0000A128A11831233270A162A
:103150008A1559088316D100831258088316D000A7
:10316000831257088316CF00831256088316CE00A9
:103170007A08D5007908D4007808D3007708D200FF
:103180000A128A1183128B250A168A157A08D10031
:103190007908D0007808CF007708CE00550883164C
:1031A000AB00831254088316AA00831253088316B7
:1031B000A900831252088316A8000A12831258210C
:1031C0000A1651088316D100831250088316D000C6
:1031D00083124F088316CF0083124E088316CE0049
:1031E0007A08D5007908D4007808D3007708D2008F
:1031F0000A128A1183128B250A168A157A08D100C1
:103200007908D0007808CF007708CE005108EA008E
:103210005008E9004F08E8004E08E7008A116F23C4
:103220008A157708E7007808E8007908E9007A0845
:10323000EA008316D100831269088316D000831236
:1032400068088316CF00831267088316CE00DB3030
:10325000D5000F30D4004930D3008030D2000A129C
:103260008A1183128B250A168A157708EB007808D5
:10327000EC007908ED007A08EE008316D500831281
:103280006D088316D40083126C088316D300831252
:103290006B088316D200D901D8013430D7008630AC
:1032A000D6000A128A11831258260A168A157A083D
:1032B000D1007908D0007808CF007708CE00DC1C58
:1032C00063298030CF0683108316D601D5013430B0
:1032D000D4008630D300831251088316DA0083129B
:1032E00050088316D90083124F088316D800831222
:1032F0004E088316D7000A128A11831247240A1631
:103300008A157708E7007808E8007908E9007A0864
:10331000EA0083106A088316D600831269088316B0
:10332000D500831268088316D400831267088316B9
:10333000D300DA01D901D8017E30D7000A128A11F0
:10334000831247240A168A157A088316D100790851
:10335000D0007808CF007708CE000A128A118312B5
:1033600011270A168A157908CC007808CB008A152F
:103370000A16532E3E08453C031DEB293030390216
:10338000EA006430F0006A08F1000A128A1102248F
:103390000A168A157808EB0030303A02EC000A3041
:1033A000F0006C08F1000A128A1102240A168A152C
:1033B00078086B07ED0030303B026D07EF00F1003D
:1033C0001430F2000A128A115C270A168A1578084E
:1033D0004A3EE400172A30303902EA006430F00037
:1033E0006A08F1000A128A1102240A168A1578085E
:1033F000EB0030303A02EC000A30F0006C08F100CB
:103400000A128A1102240A168A1578086B07ED0041
:1034100030303B026D07EF00F1001430F2000A1269
:103420008A115C270A168A157808493CE400303076
:103430003402EA000A30F0006A08F1000A128A1128
:1034400002240A168A157808EB00303035026B0723
:10345000ED00F1000A30F2000A128A115C270A1608
:103460008A1578084A3EE5003E08453C031D672A58
:1034700030303902EA006430F0006A08F1000A12C4
:103480008A1102240A168A157808EB0030303A02B5
:10349000EC000A30F0006C08F1000A128A110224D4
:1034A0000A168A1578086B07ED0030303B026D076D
:1034B000EF00F1001430F2000A128A115C270A169C
:1034C0008A150310F70C7708303EE600952A303055
:1034D0003902EA006430F0006A08F1000A128A1129
:1034E00002240A168A157808EB0030303A02EC0004
:1034F0000A30F0006C08F1000A128A1102240A1640
:103500008A1578086B07ED0030303B026D07EF003D
:10351000F1001430F2000A128A115C270A168A158B
:103520000310F70C7708393CE6003508E7003E0841
:10353000453C031DDC2A30303B020139003A031DB3
:10354000BE2A30303C02EA000A30F0006A08F1007E
:103550000A128A1102240A168A157808EB00303004
:103560003D026B07ED00F1000530F2000A128A11EE
:103570005C270A168A157808E300DB2A30303C0203
:10358000EA000A30F0006A08F1000A128A110224E7
:103590000A168A157808EB0030303D026B073C3E76
:1035A000ED00F1000530F2000A128A115C270A16BC
:1035B0008A157808E3001D2B30303B020139013CAD
:1035C000031D002B30303C02EA000A30F0006A088C
:1035D000F1000A128A1102240A168A157808EB00F3
:1035E00030303D026B07ED00F1000530F2000A12A9
:1035F0008A115C270A168A1578080B3CE3001D2BFC
:1036000030303C02EA000A30F0006A08F1000A1289
:103610008A1102240A168A157808EB0030303D0220
:103620006B07ED00F1000530F2000A128A115C27E9
:103630000A168A157808173CE30041306307E80052
:1036400030303602EA000A30F0006A08F1000A124F
:103650008A1102240A168A157808EB0030303702E6
:103660006B07ED00F1000530F2000A128A115C27A9
:103670000A168A157808E9000310690D413EE90031
:1036800030303602EA000A30F0006A08F1000A120F
:103690008A1102240A168A157808EB0030303702A6
:1036A0006B07ED00F1000530F2000A128A115C2769
:1036B0000A168A157708E3006308023C031CE90A2E
:1036C0006308023C031D692B30303802053C031CA3
:1036D000E90A6408B4006508B5006608B600670822
:1036E000B7006808BC006908BD008A150A16572E85
:1036F00020306C1E3030ED006B08F700EB1F872B7D
:10370000F709F70A7708EB002D30ED00EC176B088E
:10371000F1006430F2000A128A115C270A168A1539
:103720007708EB0030307807EE006B08F1000A30C4
:10373000F2000A128A115C270A168A1530307707C0
:10374000F00030307807EF006D08F700EC1DAA2B71
:10375000EC1F6C116C1AB72BEC1FD22B6C19D22BEF
:103760007708EE00EC18D22B7708EF00D22B303020
:103770006E02031DD22B7708EE002030ED00EC1D09
:10378000C52B6C11EC14EC1FEC1030306F02031DD4
:10379000D22B7708EF002030EE00EC1DC52BEC108B
:1037A000EC1F6C106C1DDB2B6D08F3000A128A11E4
:1037B000B9210A168A15EC1CE42B6E08F3000A12D4
:1037C0008A11B9210A168A156C1CED2B6F08F300BB
:1037D0000A128A11B9210A168A157008F3000A1212
:1037E0008A11B9210A168A1500340408F200EC1F68
:1037F000012CF217721EF20AEB09EC09EB0A03190D
:10380000EC0A6C0EF038EE00EE07E23EEF00323EBE
:10381000F1006C080F39EF07EF07F107E93EF00000
:10382000F007F0076B0E0F39F007F107F00DF10DFF
:10383000F109F10D6B080F39F107EE0D0730ED00BE
:103840000A30F107F003031C212CF007EF03031CDF
:10385000252CEF07EE03031C292CEE07ED03031CB8
:103860002D2C6D30840007307205721384037205AD
:10387000031D412C721A840A721A412C2030F70061
:103880005E2C840771300402031972170008F700D8
:10389000031D522C721B522C721A6A2CF219522CD4
:1038A00020305D2CF21F5A2C2D30F7008403721348
:1038B000F2135E2CF21572123030F707EC01040897
:1038C000EB007708F3000A128A11B9210A168A154B
:1038D0006B088400840A721F422C8A150A16352D43
:1038E0004030EB000A128A11C1210A168A153408E9
:1038F000F3000A128A11B9210A168A153508F30055
:103900000A128A11B9210A168A153608F3000A121A
:103910008A11B9210A168A153708F3000A128A118A
:10392000B9210A168A153C08F3000A128A11B92136
:103930000A168A153D08F3000A128A11B9210A16DF
:103940008A154930EB000A128A11C1210A168A151C
:103950006A08F63E0318422D0A3E452D5C1CE82CF1
:10396000C7080319E82CEB016B080A128A1184209E
:103970000A168A1500380319C52CEB0AF3000A123F
:103980008A11B9210A168A15B42C4308F3000A12C9
:103990008A11B9210A168A154408F3000A128A11FD
:1039A000B9210A168A154508F3000A128A11B921AD
:1039B0000A168A154608F3000A128A11B9210A1656
:1039C0008A156D30F3000A128A11B9210A168A1578
:1039D000422D5C1C0E2DC70803190E2D4808F3005C
:1039E0000A128A11B9210A168A154908F3000A1227
:1039F0008A11B9210A168A15EB016B080A128A117D
:103A00008B200A168A15003803190E2DEB0AF300D5
:103A10000A128A11B9210A168A15FD2C422D5C1C46
:103A20002B2DC70803192B2DEB016B080A128A11E5
:103A300095200A168A1500380319262DEB0AF30083
:103A40000A128A11B9210A168A15152D4A08EB00A7
:103A50001130EC007823422D5C1C412D0330840092
:103A60004C08EC004B08EB00F52B2F30F3000A124A
:103A70008A11B9210A168A154D08EB001330EC00A3
:103A80007823422D8A150A16E92E0A148A100A157F
:103A90008207AE2CAE2CAE2CE92CE92C0F2D0F2D6D
:103AA0002C2D2C2D2C2D84011F30830583161F14E3
:103AB0009F141F159F1107309C001C0883120D13C3
:103AC0000D308316990022309800903083129800B0
:103AD000AC01AD01C701CB01CC01CD01DC10FF3041
:103AE000DD00E00162140A128A11CB290A168A1538
:103AF0002D082C020319EA2EE001621CF82D0A128F
:103B00008A119C210A168A15E30163080A128A1198
:103B10009F200A168A1500380319962DE30AF30030
:103B20000A128A11B9210A168A15852D0A128A11DC
:103B300043230A168A15F8080319A02D0030A12D79
:103B40000130F8007818A62D6210A72D6214621CAF
:103B5000CE2D4030EB000A128A11C1210A168A15B7
:103B6000E30163080A128A11AD200A168A1500388B
:103B70000319C22DE30AF3000A128A11B9210A16A9
:103B80008A15B12D0430E300FA30E4000A128A11DC
:103B900012210A168A15E30BC42DF72D4030EB00D5
:103BA0000A128A11C1210A168A15E30163080A1252
:103BB0008A11BB200A168A1500380319E72DE30A7B
:103BC000F3000A128A11B9210A168A15D62D04307B
:103BD000E300FA30E4000A128A1112210A168A154B
:103BE000E30BE92D0A128A119C210A168A15E92E87
:103BF0000A128A1143230A168A15F808031D232E78
:103C0000EB010A128A11C1210A168A15E301630821
:103C10000A128A11C9200A168A1500380319182EAB
:103C2000E30AF3000A128A11B9210A168A15072E2F
:103C30000430E300FA30E4000A128A1112210A1655
:103C40008A15E30B1A2E0A128A118C2B0A168A1572
:103C500030303002E400F0000A30F1000A128A111C
:103C600002240A168A15303031027807E1005A081A
:103C700061020319532E6108DA000A1200280A169D
:103C80000A12332B0A160A12F92C0A168A11002876
:103C90008A150A12722F0A168A117C298A158A112E
:103CA000452E8A1500288A11E52E8A15BA295B0847
:103CB000320203198D2E5C1C8D2E0A128A11B02F30
:103CC0000A168A15F808031D882EEB010A128A11BC
:103CD000C1210A168A15E30163080A128A11D62047
:103CE0000A168A15003803197D2EE30AF3000A121A
:103CF0008A11B9210A168A156C2E0430E300FA30B5
:103D0000E4000A128A1112210A168A15E30B7F2E8B
:103D10008A115D2F8A153208DB004730EB000A124A
:103D20008A11C1210A168A15C7080319AD2E5C1C19
:103D3000AD2E4A08013C031CAD2E2130F3000A12BF
:103D40008A11B9210A168A158316061183120615DF
:103D50008316861183128611C82E5C1DB72E3F3044
:103D6000F3000A128A11B9210A168A15BE2E2030D4
:103D7000F3000A128A11B9210A168A158316061150
:103D80008312061183168611831286150430DC0611
:103D900030303202E400F0000A30F1000A128A11D9
:103DA00002240A168A157808E500303033027807B5
:103DB000F7000310F70C7708E800F1000A30F20072
:103DC0000A128A115C270A168A157708E900EA00A8
:103DD000702C1D2F6008313C0318062F0A128A111F
:103DE0009C210A168A15E30163080A128A11E3204E
:103DF0000A168A1500380319052FE30AF3000A1280
:103E00008A11B9210A168A15F42E072FE00A8316A3
:103E10008612831286163230E4000A128A111221A9
:103E20000A168A1583168612831286123230E4002F
:0E3E30000A128A1112210A168A15782D6300D3
:02400E00723FFF
:00000001FF
